:0200000480007A
:10000000B72F0000938F0F8073900F3015A8130047
:100010000000130000001300000013000000130094
:100020000000130000001300000013000000130084
:100030000000130000001300000013000000010086
:10004000970200009382020C73905230814001416C
:100050008141014281420143814301448144014580
:100060008145014681460147814701488148014950
:100070008149014A814A014B814B014C814C014D20
:10008000814D014E814E014F814F971102009381A6
:10009000A1C5170502001305E54697950300938552
:1000A000256E01461122170502001305A53C970590
:1000B0000200938525430146C52817A503001305B3
:1000C000656C97B503009385A56B37B6ABAB13068C
:1000D000B6BAD92817B103001301C16AEF503037FF
:1000E000860293D21200F512638802008242110147
:1000F0006F00001073002030824211017300203025
:10010000711116C0F3222034E3CC02FC82421101AB
:10011000130141F806C20AC40EC612C816CA1ACC88
:100120001ECE22D026D22AD42ED632D836DA3ADCC7
:100130003EDEC2C0C6C2CAC4CEC6D2C8D6CADACC97
:10014000DECEE2D0E6D2EAD4EED6F2D8F6DAFADCA7
:10015000FEDE73252034F32510340A8601A07310C7
:10016000153492402241B2414242D2426243F243AC
:10017000025492542255B2554256D2566257F25703
:10018000064896482649B649464AD64A664BF64B33
:10019000065C965C265DB65D465ED65E665FF65F83
:1001A0001301C1077300203010C16374B50011053D
:1001B000E5BF828000000000000000000000000099
:1001C000000000000000000000000000000000002F
:1001D000000000000000000000000000000000001F
:1001E000000000000000000000000000000000000F
:1001F000197106C00AC20EC412C616C81ACA1ECC8D
:1002000022CE26D02AD22ED432D636D83ADA3EDCC6
:1002100042DEC6C0CAC2CEC4D2C6D6C8DACADECC96
:10022000E2CEE6D0EAD2EED4F2D6F6D8FADAFEDCA6
:100230009702020083A2422723A02200F322103457
:1002400096DEEF00002B170102000321E125024199
:10025000F65273901234B72200009382028873A082
:10026000023082403242C2425243E24372448254DC
:100270001255A2553256C2565257E2577258864806
:100280001649A649364AC64A564BE64B764C865C1A
:10029000165DA65D365EC65E565FE65F0961730059
:1002A0002030970202009382E22523A0120023A2AD
:1002B000220023A4320023A6420023A8520023AA2E
:1002C000620023AC720023AE820023A0920223A21C
:1002D000A20223A4B20223A6C20223A8D20223AA06
:1002E000E20223ACF20223AE020323A0120523A2F2
:1002F000220523A4320523A6420523A8520523AADA
:10030000620523AC720523AE820523A0920723A2C7
:10031000A20723A4B20723A6C20723A8D20723AAB1
:10032000E20723ACF207EF40B025170102000321DA
:10033000A1170241F65273901234B7220000938243
:10034000028873A0023082403242C2425243E243EA
:10035000724482541255A2553256C2565257E25731
:10036000725886481649A649364AC64A564BE64B45
:10037000764C865C165DA65D365EC65E565FE65FB1
:10038000096173002030970202009382A21783A0B4
:10039000020003A1420083A1820003A2C20083A243
:1003A000020103A3420183A3820103A4C20183A427
:1003B000020203A5420283A5820203A6C20283A60B
:1003C000020303A7420383A7820303A8C20383A8EF
:1003D000020403A9420483A9820403AAC20483AAD3
:1003E000020503AB420583AB820503ACC20583ACB7
:1003F000020603AD420683AD820603AEC20683AE9B
:10040000020703AFC20983AF820782807370043092
:10041000197106C00AC20EC412C616C81ACA1ECC6A
:1004200022CE26D02AD22ED432D636D83ADA3EDCA4
:1004300042DEC6C0CAC2CEC4D2C6D6C8DACADECC74
:10044000E2CEE6D0EAD2EED4F2D6F6D8FADAFEDC84
:100450009702020083A2420523A0220086DEEF203D
:10046000402D17010200032121040241F65273902E
:100470001234B72200009382028873A002308240B7
:100480003242C2425243E243724482541255A25550
:100490003256C2565257E257725886481649A649F4
:1004A000364AC64A564BE64B764C865C165DA65DD0
:1004B000365EC65E565FE65F09617300203073707A
:1004C000043001A07310453082807325403073F0F2
:1004D00043308280970700009387A7FE232EB5FE46
:1004E0002322C5FA232635F82320F5F8130505F84D
:1004F0008280411106C6EF40D005EF10700901E57A
:10050000B24041018280B24041016F2080229307B6
:1005100085007D575CC118C55CC51CC9232005003A
:1005200082802328050082805C41DCC1984798C501
:1005300098474CC38CC788C91C4185071CC1828061
:100540009041FD57130785006314F60039A83E87D4
:100550005C439443E37DD6FEDCC18CC798C54CC395
:1005600088C91C4185071CC1828018495C43EDB7CE
:10057000584114451C4914C71845544154C3D84325
:100580006314A7001845D8C32328050088437D15A8
:1005900088C382803041AE8701CE4C455841B29528
:1005A0004CC563E4E5000C414CC53E856F30101F1F
:1005B0008280411122C406C62A8426C2EF209010F0
:1005C0003C44635BF0025C5085CB9304440209A871
:1005D0003C44FD173CC43C446350F0025C5089CF5E
:1005E0002685EF20A0566DD5EF2080763C44FD1780
:1005F0003CC43C44E344F0FEFD573CC4EF20D00E25
:10060000EF20500C7C40635BF0021C4885CB9304C8
:10061000040109A87C40FD177CC07C406350F002B7
:100620001C4889CF2685EF2060526DD5EF2040729F
:100630007C40FD177CC07C40E344F0FEFD577CC04D
:100640002244B240924441016F20100A29C5411151
:1006500022C426C22A8406C6AE84EF20B0063440E7
:100660005C5C1840232C0402B387F6027D5670C0F0
:1006700018C430C4B386D740BA9736975CC058C404
:1006800091EC1C489DE3EF203006B2402244924496
:100690000545410182807370043001A013050401F7
:1006A000BD3513054402A535F9BF13050401EF203C
:1006B000E0498547E319F5FC913BF1B701E573701B
:1006C000043001A0011126CA4AC84EC606CE22CC6B
:1006D000B2892E89AA84A5C53305B502130555052F
:1006E000EF3080732A8435C1930745051CC144DC73
:1006F00023202405EF20007D34405C5C18407D56AB
:10070000B387F602232C040270C018C430C413054A
:100710000401B386D740BA9736975CC058C4C53B2E
:1007200013054402ED33EF20207C23083405228595
:10073000F2406244D2444249B249056182801305C5
:100740004005EF30606D2A8401E57370043001A02C
:1007500000C071BF01E57370043001A06375B5007E
:100760007370043001A0411122C409462E848145D2
:1007700006C6A93711C500DDB2402244410182807E
:100780007370043001A05D7186C6A2C4A6C2CAC03F
:100790004EDE52DC56DA5AD85ED632C6630A051CE3
:1007A0006382051C89476399F600585D8547630598
:1007B000F7007370043001A03689AE842A84EF20DC
:1007C000A05B11E5B24781C77370043001A0EF2030
:1007D000606F185C5C5C014B894BFD59130A040186
:1007E000930A44026365F70C63077919B247638182
:1007F000072463150B002808EF206048EF20C06E27
:10080000EF10C04FEF20006C7C406394370123222F
:1008100004043C446394370123240404EF20C06C97
:100820006C002808EF20C047631E051EEF2080697A
:10083000185C5C5C630CF70AEF20006BEF208068AB
:100840003C44634FF00039A85685EF20203019C191
:10085000EF2000503C44FD173CC43C446354F0007E
:100860005C50FDF323243405EF200068EF20806501
:100870007C40634FF00039A85285EF20202D19C12C
:10088000EF20004D7C40FD177CC07C406354F0009D
:100890001C48FDF323223405EF200065EF10006BA8
:1008A000054BEF202062185C5C5CE37FF7F2304080
:1008B0006305060C631F09120844A685EF30006E1D
:1008C0001C4434405840B6971CC463EAE70A1C5CD9
:1008D00014405850850714C41CDC5DC7130544023E
:1008E000EF20C02685476311F50AC9A8EF20C05F35
:1008F000B2455285EF204007EF20C05C3C44634F77
:10090000F00039A85685EF20602419C1EF2040443B
:100910003C44FD173CC43C446354F0005C50FDF380
:1009200023243405EF20405CEF20C0597C40634F06
:10093000F00039A85285EF20602119C1EF20404115
:100940007C40FD177CC07C406354F0001C48FDF3E4
:1009500023223405EF204059EF10405F31F17D3400
:10096000054B81B73C41E38F07E27370043001A06F
:100970007370043001A0304021E61C4085C71C5C28
:10098000585085071CDC39FBEF2000560545B64062
:10099000264496440649F259625AD25A425BB25BE7
:1009A000616182804840EF2040491C5C58502322FE
:1009B000040085071CDCE31307F279D5813CE9B715
:1009C0004844A685EF30805D3C4058441440B3074E
:1009D000F0403E9758C4637CD7025840BA975CC435
:1009E00009475C506306E902185C050718DCC9DF9B
:1009F000F5B54844A685EF30605A3C405844144051
:100A0000B307F0403E9758C4E37CD7FCF9B75C507D
:100A1000185C79DB185C7D1718DC185C050718DC9E
:100A2000A5D76DBD22857136EF104052014585B7BF
:100A3000EF20804B0145A1BF411126C2AA841305B6
:100A4000400522C406C6EF30203D2A8415CD232C54
:100A50000502FD577CC10547410558DC3CC42322F3
:100A60000400232004002324040023260400232060
:100A7000040423089404613C13054402493C814664
:100A800001468145228501332285B24022449244A9
:100A9000410182800DC5411122C426C206C64AC04A
:100AA000032945002A84EF20602C8144630CA900AF
:100AB000B2402244268502499244410182807370EB
:100AC000043001A05C448544FD175CC4F5F3814605
:100AD0000146814522854539E1BF31CDA1C90111CA
:100AE00022CC26CA4AC852C406CE4EC68947B6840E
:100AF00032892E8A2A846399F600585D8547630FF0
:100B0000F7047370043001A0C932185C5C5CAA89D8
:100B10006366F70281444E857532F2406244268551
:100B20004249D244B249224A056182803C41C5DB38
:100B30007370043001A07370043001A0304041E2B2
:100B40001C40D5CB1C5C7D5785071CDC3C4463876F
:100B5000E7083C44854485073CC475BFBD32185C3A
:100B60005C5CAA89636DF702304079DA4844D2852B
:100B7000EF30C0423C4058441440B307F0403E9729
:100B800058C46375D7005840BA975CC48947E39B43
:100B9000F4FA1C5CC5DB1C5CFD171CDC65B730403F
:100BA00045D24844D285EF30603F3C405844144021
:100BB000B307F0403E9758C4E367D7FCD9BFDDF4D4
:100BC0000844D285EF30803D1C4434405840B697ED
:100BD0001CC4E3E9E7F61C401CC4ADB75C50854477
:100BE0009DDB13054402EF10707615D5E30509F27D
:100BF000232099000DB74840EF2020242322040031
:100C000091B721CD3C4181C77370043001A01C41D4
:100C1000A1CB011122CC26CA2A844AC84EC606CED0
:100C20002E896530185C5C5CAA898144637DF7007D
:100C30001C5C7D5785071CDC3C446388E7023C4410
:100C4000854485073CC44E85B538F240624426850C
:100C50004249D244B249056182807370043001A0D8
:100C60005C41C5DB7370043001A05C5099E385449E
:100C7000D9BF13054402EF10706D75D9E30909FE61
:100C800085472320F900E5B7397106DE22DC26DA34
:100C90004AD84ED652D456D232C66302051C638A55
:100CA000051AB68AAE892A84EF20000D11E5B247F5
:100CB00081C77370043001A0EF20C0201C5C6392D8
:100CC0000714B247638E070A2808EF10507BFD54C3
:100CD00013094402130A0401EF200021EF1000025F
:100CE000EF20401E7C4063949700232204043C4480
:100CF0006394970023240404EF20001F6C0028084D
:100D0000EF10107A63130518EF20C01B1C5CADCFE9
:100D1000EF20801DEF20001B3C44634FF00039A8FA
:100D20004A85EF10B06219C1EF2080023C44FD17E4
:100D30003CC43C446354F0005C50FDF324C4EF20F9
:100D4000A01AEF2020187C40634FF00039A852858C
:100D5000EF10D05F19C1EF10B07F7C40FD177CC051
:100D60007C406354F0001C48FDF364C0EF20C017C2
:100D7000EF10C01DEF2000151C5CC1E7B247A9FFB2
:100D8000EF208016014555A0EF2000161C40DDC75E
:100D9000B2454A85EF10503DEF20C0123C44634FEE
:100DA000F00039A84A85EF10705A19C1EF10507A37
:100DB0003C44FD173CC43C446354F0005C50FDF3DC
:100DC00024C4EF206012EF20E00F7C40634FF0005E
:100DD00039A85285EF10905719C1EF1070777C40F9
:100DE000FD177CC07C406354F0001C48FDF364C0D8
:100DF000EF20800FEF10801531C9EF20A00C1C5C94
:100E0000B5DFCE8522854444EFF0CFF8639C0A0419
:100E10001C5C1840FD171CDC01E7EF20601148C086
:100E20001C48A1EFEF20400C0545F2506254D2540B
:100E30004259B259225A925A21618280EF20800889
:100E40004840EF107075EF20200A99B7EFF00FDCE3
:100E50006DB73C41E38707E47370043001A0737001
:100E6000043001A05C5044C4D5DF13054402EF10E8
:100E7000F04D4DD9EFF08FD975B713050401EF1080
:100E8000F04C8547E310F5FAF5B72285EFF06FF2E5
:100E9000EF10C00B014551BF1DC9411122C44AC00A
:100EA00006C626C244412E892A84EF10306C638323
:100EB000A40281464A8681452285F933854763002D
:100EC000F502B2402244924402494101828073708B
:100ED000043001A05C44054585075CC4DDB75C4473
:100EE00085075CC4F9BF15CDADC9011122CC26CA56
:100EF0004AC84EC652C42A8406CE3289AE89EFF063
:100F0000CFDC1C5C2A8A814485E35285EFF08FDBBD
:100F1000F240624426854249D244B249224A0561E0
:100F200082807370043001A0304001CE4C445C409C
:100F3000B2954CC463E4F5000C404CC44E85EF30D0
:100F4000E0051C5C7D57FD171CDC7C40638CE700D2
:100F50007C40854485077CC04DBF3C41D9D7737028
:100F6000043001A01C4899E3854445B713050401EA
:100F7000EF10D03D75D9E30909FE85472320F9001C
:100F8000E5B721C93C41A1CDA1CB011122CC26CA94
:100F90004AC852C42A8406CE4EC62E8AEFF0EFD23B
:100FA0001C5C2A89814491CB8329C400D285228587
:100FB000EFF04FDE8544232634014A85EFF08FD0D1
:100FC000F240624426854249D244B249224A056130
:100FD00082807370043001A07370043001A0EDDFD3
:100FE0007370043001A001E57370043001A0411159
:100FF00022C42A8406C6EF10F06C005CEF10D06E9D
:10100000B240228522444101828001E573700430A0
:1010100001A0411106C622C42A84EF10B06A1C5CEC
:10102000405C1D8CEF10506C2285B240224441017F
:10103000828019C1085D82807370043001A01DCDCB
:101040009787030093870770D843630CE502D8475E
:10105000630CE504D84B6307E504D84F6302E5044D
:10106000D853630DE502D8576308E502D85B6303E4
:10107000E502D85F630EE5006F20306C73700430BA
:1010800001A001470E07BA9723A007006F20F06A5E
:101090001D47CDBF1947FDB71547EDB71147DDB760
:1010A0000D47CDB70947F9BF0547E9BF68458280BD
:1010B0006CC5828003450505828009C5085D13352E
:1010C000150082807370043001A019C51C5D485D55
:1010D0001D8D1335150082807370043001A0978731
:1010E000030093872766984305C3984705C7984B25
:1010F00005C7984F05C7985305C7985705C7985B0C
:1011000015C7985F15C3828001470E07BA978CC335
:10111000C8C382800547D5BF0947C5BF0D47F5B78E
:101120001147E5B71547D5B71D47C5B71947F1BFF3
:101130009787030093870761D8436308E502D84780
:10114000630BE502D84B630AE502D84F6309E50259
:10115000D8536308E502D8576307E502D85B6308F4
:10116000E502D85F6303A702828001470E07BA97A2
:1011700023A0070082800547D5BF0947C5BF0D479B
:10118000F5B71147E5B71547D5B71D47C5B7194797
:10119000F1BF411122C426C24AC02A8406C6AE84C9
:1011A0003289EF1030527840FD576314F700232244
:1011B00004043844FD576314F70023240404EF109B
:1011C000B0521C5C99E74A86A68513054402EF10CD
:1011D000B00CEF10304F3C44635BF0025C5085CBA9
:1011E0009304440209A83C44FD173CC43C446350AA
:1011F000F0025C5089CF2685EF1050156DD5EF10A9
:1012000030353C44FD173CC43C44E344F0FEFD57FC
:101210003CC4EF10704DEF10F04A7C40635BF0026D
:101220001C4885CB9304040109A87C40FD177CC0B1
:101230007C406350F0021C4889CF2685EF101011C6
:101240006DD5EF10F0307C40FD177CC07C40E3444E
:10125000F0FEFD577CC02244B24092440249410155
:101260006F10904805C579714ECE52CC06D63E8A95
:1012700022D426D24AD056CA5AC85EC662C4A547EE
:10128000BA8963F8E7007370043001A0737004300A
:1012900001A0AA8AAE843289B68B428B63090822E8
:1012A00013050006EF2050372A84630D05200A0934
:1012B000232865034A869305500A5A85EF20105C5F
:1012C00003C704001C587119230AE40203C7040071
:1012D0003E991379C9FF79C783C71400A30AF402A2
:1012E00083C71400E1C383C72400230BF40283C720
:1012F0002400CDCB83C73400A30BF40283C7340092
:10130000D5C383C74400230CF40283C74400D9CB60
:1013100083C75400A30CF40283C75400C1C783C71A
:101320006400230DF40283C76400ADCF83C774004B
:10133000A30DF40283C77400B5C783C78400230ECE
:10134000F40283C78400B9CF83C79400A30EF402CC
:1013500083C79400A1CB83C7A400230FF40283C7E3
:10136000A400A9C383C7B400A30FF40283C7B400C9
:1013700095CB83C7C4002300F40483C7C4009DC376
:1013800083C7D400A300F40483C7D40081CF83C7EC
:10139000E4002301F40483C7E40089C783C7F40091
:1013A000A301F404130B44005A85A301040423266B
:1013B000340323283405232A0404EFF08F96130501
:1013C0008401EFF00F96A947B3873741232C04041B
:1013D00000C81CCC40D023220404232E04045E86C3
:1013E000D6854A85EFF00F8F08C063040A002320DA
:1013F0008A007370043017F9010013092909832743
:10140000090097F401009384240A91C798409C40F6
:101410007C4385077CC317F701001307E7071C43CC
:10142000850797F6010023A9F6069C40D5CB8327B4
:10143000090017FA0100130AAA1489EB9C40DC5733
:1014400063E6F90097F7010023A0870697F70100EC
:101450009387C702984397F60100938666035C540E
:101460009442050717F60100232AE60038C463F604
:10147000F60017F70100232DF7005147B387E70265
:10148000DA853305FA00EFF02F8A8327090081C738
:101490009C40FC43BDE383270900054499C79C4059
:1014A000DC5763F43701EFE07FF62285B250225417
:1014B00092540259F249624AD24A424BB24B224CF0
:1014C000456182805A85EF2050277D54F9BF13155E
:1014D0002600EF2070142A8BE31405DC7D54F1B74D
:1014E00097F7010023A287FC184385476301F702A1
:1014F00017FA0100130ACA0891BF984094407C4330
:10150000FD177CC3FC42C1FB7360043069B7814A9C
:1015100017FA0100130ACA06514CA94B33858A03F6
:10152000850A5295EFE0BFFEE39A7AFF97FB010030
:10153000938B8B115E85EFE09FFD97FA0100938AF4
:10154000EA115685EFE0BFFC17F5010013054512BF
:10155000EFE0FFFB17F501001305C512EFE03FFBBD
:1015600017F5010013054513EFE07FFA97F7010027
:1015700023AA77F397F7010023A457F3C1BD4111C4
:1015800022C406C626C24AC02A847370043097F467
:1015900001009384A4EF9C40F9E311E497F7010064
:1015A000938787F08043130944004A85EFE05FFC8E
:1015B0001C5489C713058401EFE09FFBCA8517F50A
:1015C00001001305250CEFE03FF697F70100938724
:1015D000E7EC984397F70100938747EA9C43050798
:1015E00097F6010023ACE6EA9840850797F60100DC
:1015F00023A6F6E801CB97F701009387E7EA984323
:10160000784349EF9C40B1C797F701009387C7E93A
:101610009843630F870873700430984039EB17F7CD
:101620000100130727E814439442A5E27D5797F67B
:10163000010023A3E6E4984009CF9843784311CBF7
:10164000984394437C43FD177CC3FC4299E3736049
:101650000430B2402244924402494101828097F70B
:101660000100938767E498439C437C4385077CC3D0
:101670002DB794439843F8420507F8C217F70100C5
:10168000130747E214439442D5D2184358475847AA
:10169000584397F6010023A1E6DE71BF98439443B7
:1016A0007C43FD177CC3FC42B1FF7360043099BFDB
:1016B00097F70100938707DC9C4381C77370043060
:1016C00001A02244B2409244024941016FE01FD47C
:1016D00041C517F70100130727DD14438147638BCA
:1016E000A606411106C622C426C27370043097F6BE
:1016F00001009386A6D99C4291C710431C437C42AB
:1017000085077CC29C42AA84404981C71C43FC4394
:10171000B9E797F701009387E7D89C43638B870469
:1017200097F701009387C7D79C436384870497F793
:101730000100938767F66309F40297F70100938726
:1017400067F46301F4028547B240224492443E8527
:10175000410182803E8582807370043001A0EF4099
:10176000604445BF9147CDB79C5493B71700890794
:10177000E1BF8947D1BF7370043097F701009387A9
:10178000E7D0984309EF15C59C43485581CB97F79F
:101790000100938767D19843784315E3828017F758
:1017A0000100130767D014431843F8420507F8C235
:1017B00061FD17F70100130727CF0843F1B79843DE
:1017C00094437C43FD177CC3FC42E9FB7360043007
:1017D0008280411122C42A8406C6EFE01FCF11E4A3
:1017E00097F70100938747CC80434054EFE09FCDAB
:1017F000B2402285224441018280A54763F5B700AB
:101800007370043001A0011122CC06CE26CA4AC84A
:101810004EC652C42A847370043017F901001309AC
:10182000E9C683270900D5EF79C43C486389F508E8
:1018300017F70100130747C763FCB7001443638D14
:10184000860C18434457B3B4950093C4140029A0E0
:101850000443818C93B4140058546384E70A1C4CED
:101860002CC863C60700A947B385B7400CCC9317B3
:101870002700BA97584897F90100938969D08A07D9
:10188000CE97631BF702130A44005285EFE05FCE48
:1018900017F701001307C7BF5C5418436376F700BE
:1018A00017F701002326F7BE5147B387E702D28519
:1018B0003385F900EFE05FC799C0EFE03FB58327BC
:1018C000090081CB97F70100938707BE9C43FC4337
:1018D0009DEBF2406244D2444249B249224A05613A
:1018E000828097F70100938727BC98439C437C43F1
:1018F00085077CC31DF897F701009387E7BA8043FB
:101900002DB74CD4A9BF6244F240D2444249B249F7
:10191000224A05616F40002981443DBF25C1011164
:1019200026CA97F40100938424B89C4006CE22CCAA
:101930004AC84EC6638DA7027370043017F90100C0
:101940001309C9B48327090091C798409C407C4380
:1019500085077CC3584997F701009387E7D3630253
:10196000F7028327090081C79C40FC43A5EBF240A6
:101970006244D2444249B2490561828073700430A6
:1019800001A01C5517F70100130787CEE38BE7FC76
:10199000E9FB930945002A844E85EFE07FBD17F7E8
:1019A00001001307E7AE5C5418436376F70017F79E
:1019B0000100232FF7AC5147B387E70217F5010069
:1019C000130505BCCE853E95EFE01FB69C405854EC
:1019D000DC57E368F7F8EFE07FA361B76244F240B9
:1019E000D2444249B24905616F40C01B15CD011177
:1019F00022CC26CA4AC82A8406CE4EC6EFE0FFACE7
:101A0000584897F70100938727C92A8981446300C2
:101A1000F7024A85EFE01FABF24062442685424957
:101A2000D244B249056182807370043001A01C5415
:101A300017F501001305C5C3E38DA7FCF9FB97F764
:101A40000100938727A39C43A9EB97F70100938795
:101A5000A7A59C43445493094400DC574E85B3B476
:101A6000F400EFE0FFB017F70100130767A25C5422
:101A7000184393C414006376F70017F70100232975
:101A8000F7A05147B387E70217F50100130545AFEB
:101A9000CE853E95EFE05FA9ADBF93058401EFE0F1
:101AA000BFA885BF0111056506CE22CC26CA4AC84B
:101AB0004EC652C456C25AC0EF200036630E051AF5
:101AC000AA8413050006EF2020352A84630A051C2A
:101AD00005669305500A04D92685EF20205A04583C
:101AE0008567F117BE94B7474C4593879744130A0F
:101AF00044005CD85285230C0402A301040423266D
:101B0000040223280404232A0404EFE09FA1130500
:101B10008401EFE01FA1A947232C0404F19800C819
:101B20001CCC40D023220404232E04040146971524
:101B300000009385E5B12685EFE0DF9908C073705A
:101B4000043017F90100130969948327090097F4F9
:101B500001009384649591C798409C407C4385071D
:101B60007CC317F70100130727931C43850797F6DB
:101B7000010023A3F6929C40C9C38327090097F96B
:101B800001009389E99F81EB9C40DC5789E797F737
:101B9000010023AB879097F701009387278E984326
:101BA00097F601009386C68E5C549442050717F69B
:101BB00001002325E68C38C463F6F60017F7010010
:101BC0002328F78C139527003E950A05D2854E955C
:101BD000EFE09F958327090081C79C40FC43DDE728
:101BE0008327090091C39C40EF1070498547630526
:101BF000F50C59E17370043001A097F7010023A59B
:101C0000878A1843854797F9010093896997E314F8
:101C1000F7F8CE8A17FB0100130B0BA35685D10AE8
:101C2000EFE0FF8EE31C5BFF17F501001305C5A174
:101C3000EFE0FF8D97FA0100938A4AA25685EFE004
:101C40001F8D17F501001305A5A2EFE05F8C17F5B6
:101C50000100130525A3EFE09F8B17F50100130585
:101C6000A5A3EFE0DF8A97F7010023AD678397F71D
:101C7000010023A7578305B7F2406244D24442498A
:101C8000B249224A924A024B0561828098409440B0
:101C90007C43FD177CC3FC42A1F77360043089B715
:101CA0006244F2404249B249224A924A024B268596
:101CB000D24405616F20602873700430FD5717E728
:101CC0000100232BF77A624497E7010023A0A77C49
:101CD000F240D2444249B249224A924A024B97E723
:101CE000010023A9077A05616FE0AFDB7370043050
:101CF00097E7010023AC07786FE0EFE817E70100F2
:101D0000130747771C4385071CC382807370043018
:101D100097E7010093878777984305E317E701006A
:101D20001307477708439C4381CB97E701009387CC
:101D3000A7779843784301EF828017E701001307E4
:101D4000A77614431843F8420507F8C2C1BF984369
:101D500094437C43FD177CC3FC42F9FF736004305D
:101D60008280411106C622C4EFE02FF697E70100FA
:101D7000938747728043EFE0EFF4B240228522441C
:101D80004101828097E70100938707718843828031
:101D9000797106D622D426D24AD04ECE52CC56CA1B
:101DA0005AC85EC697E701009387C76C9C43B1EFA2
:101DB00017E701001307076E1C43850797E601002C
:101DC00023AAF66C832A0700638F0A0697E70100AF
:101DD0009387876A9C43814463F1FA0897E901007D
:101DE0009389097A17EA0100130A0A6C83270A000B
:101DF0008546D85793172700BA978A07BE9983A7B5
:101E0000090063FFF600854421A897E70100938746
:101E1000A7679C438144850717E701002326F766DF
:101E200097E70100938707669C4391C38544B250AE
:101E30002254268502599254F249624AD24A424BB0
:101E4000B24B4561828017E401001304A4651C4075
:101E50009C43DDC37370043001A017E40100130438
:101E6000646497E901009389A97117EA0100130AD4
:101E7000AA6317EB0100130BAB611C409C43B5C375
:101E80001C40DC4703A9C70083274900930B490086
:101E90005E8563EEFA04EFE0AFED83278902130558
:101EA000890199C3EFE0CFEC8327C90203270B0018
:101EB000DE85139527003E950A054E956376F7005B
:101EC00017E701002326F75CEFE00FE683270A00FF
:101ED0000327C902DC57E362F7FA1C4085449C43A0
:101EE000C5F3FD5717E701002328F75801B717E797
:101EF00001002323F758DDBD17E701001307475AF8
:101F00001C40184397E6010023AEE65817E701008E
:101F10002328F75897E70100938787569C43850746
:101F200017E70100232EF7541C409C4399E7FD5707
:101F300017E701002322F75451BD1C40DC47DC4762
:101F4000DC4317E701002329F75249B597E7010061
:101F500093874752984301E77370043001A0011141
:101F600006CE22CC26CA4AC84EC652C456C25AC051
:101F70007370043097E4010093844451984061EBFE
:101F800098437D1797E6010023A6E64E9C43D9EBC4
:101F900097E70100938747509C43C9C797EA010020
:101FA000938A0A5E17EA0100130A8A4E17E90100B4
:101FB0001309894F854919A83385EA00EFE0CFD688
:101FC000832709005854DC576379F70483A70A0F65
:101FD000C1CF83A7CA0FC04713058401EFE04FD9D3
:101FE000130B44005A85EFE0AFD85C5483260A00F7
:101FF000DA85139527003E950A052A875695E3FD55
:10200000F6FA17E701002325F748EFE0EFD1832721
:1020100009005854DC57E36BF7FA97E7010023A354
:1020200037476DB701449C4081CB97E70100938708
:10203000A7479C43FC4395E72285F2406244D24483
:102040004249B249224A924A024B0561828017E70F
:1020500001001307674514431843F8420507F8C207
:1020600005B7EF303034C9BF17E401001304C44191
:102070001C4095C31C40054999CF193B09C597E7FA
:10208000010023A127411C40FD1717E70100232D64
:10209000F73E1C40FDF397E701009387A73E984366
:1020A0008547E311F7F8EFE06FB60544ADBF11CDFA
:1020B00081E57370043001A017E701001307873B27
:1020C0001C4399C77370043001A07370043001A0E1
:1020D000411122C406C614431841850617E60100C3
:1020E000232AD63897E601009386C63A94423304F1
:1020F000B70000C163F7E602637FE40063FD86007A
:1021000097E701009387473A88431105EFE04FC6F0
:102110002285EF30F0221D3D01C9B2402244410129
:102120008280E36FE4FCD9BF2244B24041016FE0FA
:10213000EFAD11C917E701001307C7331C4391C75F
:102140007370043001A06FE06FAC411106C622C469
:102150001843AA87050797E6010023ADE63097E606
:1021600001009386663417E701001307A73218436E
:1021700088423304F7001105EFE08FBF2285EF306E
:10218000301CE93311E52244B24041016FE00FA851
:10219000B240224441018280411122C406C697E721
:1021A00001009387272D9C430144850717E7010011
:1021B0002322F72C97E701009387072E9C4363E0C7
:1021C000F51217EE0100130E6E4797E2010093829D
:1021D000623A01440147854F1303500A21A0311E82
:1021E000638DC20B83278EFFBA86F5DB8327CEFF74
:1021F000DC43232EFEFE638AC70F03AFC700DC4318
:102200002A97814E232EFEFE6385C70783A8C70049
:1022100093874803232017015CC383A788042326E0
:10222000F7011CC783A7C8021CCB83A70805232C72
:1022300007005CCB03A8080383470800639067048A
:10224000C287850783C60700B3850741E38B66FE17
:102250008981C205C181231EB700850E13070702BD
:1022600063061F038327CEFFDC43232EFEFEE39F7E
:10227000C7F983274E00232EFEFE49BF8145231E4A
:10228000B700850E13070702E31E1FFD7694131790
:102290005400311EBA86E397C2F597E70100938791
:1022A000672003AE070083270E00639D070E97E7A4
:1022B00001009387E71E03AE070083270E00639299
:1022C000071817EE0100130EAE2B83274E109DE367
:1022D00083278E116395072019C223200600BD3184
:1022E0002285B24022444101828083274E00232E62
:1022F000FEFE21B783278E1017EF0100130F0F3951
:10230000DC4317E701002321F7386380E73383A21A
:10231000C700DC43AA96814E17E701002326F73653
:10232000914F1303500A6388E70783A8C700938778
:10233000480323A01601DCC283A7880423A6F60164
:102340009CC683A7C8029CCA83A7080523AC0600C5
:10235000DCCA03A80803834708006391672AC28781
:10236000850703C70700B3850741E30B67FE93D7D3
:102370002500C207C183239EF600850E93860602C0
:102380006386122983278E10DC4317E70100232D73
:10239000F72EE39CE7F983270E1117E701002325A9
:1023A000F72E61B783274E00130F8E00D4432322EC
:1023B000DE006388E629B307E500D84283A2C600A1
:1023C000814E2322EE00894F1303500A6306EF0665
:1023D0008328C7001387480323A01701D8C303A786
:1023E000880423A6F70198C703A7C80298CB03A7C0
:1023F000080523AC0700D8CB03A80803034708004F
:102400006318671C4287050783460700B305074129
:10241000E38B66FE13D7250042074183239EE70026
:10242000850E93870702638D121B83264E00D842C8
:102430002322EE00E31EEFF80327CE002322EE0056
:1024400041BF83274E00130F8E00DC432322FE0082
:102450006384E71F83A2C700DC43AA96814E232230
:10246000FE00894F1303500A6306FF0683A8C700C6
:102470009387480323A01601DCC283A7880423A600
:10248000F6019CC683A7C8029CCA83A7080523AC93
:102490000600DCCA03A80803834708006396671098
:1024A000C287850703C70700B3850741E30B67FEB3
:1024B00093D72500C207C183239EF600850E93861D
:1024C0000602638B120F83274E00DC432322FE009B
:1024D000E31EFFF88327CE002322FE0041BF83279F
:1024E000CE1197EE0100938EAE1BDC4317E701007F
:1024F0002326F71A6384D71383AFC700DC4333075F
:10250000D500014397E6010023AAF6180D4F894232
:102510009308500A6387D707C8479307450308C342
:102520005CC33C452326E7011CC75C551CCB1C55EE
:1025300099C3232657003C49232C07005CCB032872
:1025400005038347080063951705C287850783C67F
:102550000700B3850741E38B16FF93D72500C20719
:10256000C183231EF700050313070702638AAF0226
:102570008327CE11DC4397E6010023A1F612E39DE9
:10258000D7F983274E1297E6010023A9F61069B701
:102590008147231EF700050313070702E39AAFFCE8
:1025A0001A94E31C06D225BB8147239EF600850EB4
:1025B00093860602E39912F117EE0100130E4EFC0A
:1025C00083274E10769493165400E38307D01DB3EF
:1025D0000147239EE700850E93870702E39712E5E4
:1025E00097E701009387C7EB03AE07007694931635
:1025F000540083270E00E38607CCA1B58147239EB4
:10260000F600850E93860602E39E12D783278E116D
:10261000769493165400E38107CCD1B583274E12EC
:1026200017E70100232CF706C1BD83270E1117E71A
:102630000100232BF704E1B98327CE002322FE00FB
:1026400011BD8326CE002322DE00B5B3797126D2D8
:102650004AD04ECE52CC56CA5AC85EC606D622D4EE
:1026600097E90100938909E117E90100130949F18C
:1026700017EA0100130A8AE197EA0100938ACAE285
:1026800097EB0100938B4BE197E40100938404E105
:10269000054B21A883A7090003244910850717E7E4
:1026A00001002329F7DC5D3011E89C40E5F7832722
:1026B0000900E37CFBFEEFD07FD5C5BF737004300B
:1026C00083270A00B9E383270911C0471305440093
:1026D000EFD01FEA83A70B00FD1717E70100232D9A
:1026E000F7DA9C40FD1717E701002329F7DA832763
:1026F0000A0089C783A70A00FC4385E30858EF1046
:10270000D0032285EF1070034DB703A70A0083A7FB
:102710000A007C4385077CC37DB703A70A0083A614
:102720000A007C43FD177CC3FC42E9FB7360043064
:10273000F1B797E701009387E7D39C43DDE34111AD
:1027400006C697E7010023AF07D217E7010013077A
:10275000A7D51C43B7A6A5A59386565A9C5B8C4368
:10276000639BD500D0436318B60094476395C600B9
:10277000DC476388D70008430C4393854503EF206B
:10278000C07697E601009386A6D0904217E7010035
:10279000130707DF11A89C42B9CB9C42FD1717E62F
:1027A00001002327F6CE904293172600B2978A079E
:1027B000BA979C43EDD3904293172600B2978A07AD
:1027C000B305F700D441A107BA97D442D4C16383BB
:1027D000F602DC46B24017E701002327F7CC41019F
:1027E0008280854717E70100232EF7C88280737027
:1027F000043001A0D1473306F602D442329754C3C5
:10280000C9BF01114AC806CE22CC26CA4EC62A89A3
:102810007370043097E40100938444C79C4017E42C
:102820000100130464C8D9E76314090003290400F4
:10283000930949004E85EFD0BFD38327890289C70A
:1028400013058901EFD0DFD2CE8517E5010013050E
:10285000A5E4EFD07FCD9C4081C71C40FC43ADE395
:102860001C40638B27079C409DCF737004309C40B5
:10287000C1EB97E701009387E7C29843184325EB24
:10288000FD5717E701002329F7BE9C4089CF1C4064
:10289000FC4391CB184014407C43FD177CC3FC42A1
:1028A00099E373600430F2406244D2444249B24931
:1028B0000561828018401C407C4385077CC3ADB70E
:1028C000184014407C43FD177CC3FC42D1FB73606D
:1028D00004301C40E39927F99C40A1C397E701000D
:1028E000938747B99C43ADCB7370043001A09C43E0
:1028F000DC47DC47DC4317E70100232FF7B671B74D
:1029000018401C407C4385077CC397E701009387F0
:1029100067B9984318432DD7D9BF97E7010093872C
:10292000A7B717E701001307A7C59C430327871123
:10293000631DF700F240624497E7010023A607B643
:10294000D2444249B249056182806244F240D24495
:102950004249B2490561F1BB6244F240D244424966
:10296000B24905616FD09FAA3DC9411126C297E4C3
:102970000100938464B34AC02E898C4006C622C4E9
:10298000E105EFD0FFBB88401105EFD07FBEFD57BA
:10299000630AF90497E701009387C7AF8043984023
:1029A0009C434A9440C3636CF40497E70100938707
:1029B00067AF88438C409105EFD09FB897E701003F
:1029C000938787AB9C436376F40097E7010023A5C8
:1029D00087AAB24022449244024941018280737026
:1029E000043001A08C402244B2409244024917E5D1
:1029F0000100130565CA910541016FD0FFB297E749
:102A000001009387E7A9884322448C40B240924456
:102A10000249910541016FD0BFB211C997E701008A
:102A2000938747A59C4399E77370043001A07370A6
:102A3000043001A0411126C297E401009384C4A68A
:102A40009840AE878C40B7060080D58F06C622C45A
:102A50001CCFE1053284EFD03FAD88401105EFD0A7
:102A60003FB1FD57630EF40097E70100938787A2FB
:102A70008843B24092442295224441016F30400C79
:102A80008C402244B240924417E501001305C5C0B2
:102A9000910541016FD05FA925CD411126C297E470
:102AA0000100938464A04AC02E898C4006C622C4CB
:102AB000E1053284EFD05FA788401105EFD05FAB0E
:102AC0008547630AF40497E701009387A79C804336
:102AD00098409C434A9440C3636CF40497E7010018
:102AE0009387479C88438C409105EFD07FA597E75B
:102AF0000100938767989C436376F40097E7010091
:102B000023AC8796B240224492440249410182801C
:102B10007370043001A08C402244B24092440249B8
:102B200017E50100130545B7910541016FD0DF9FFF
:102B300097E701009387C796884322448C40B240B0
:102B400092440249910541016FD09F9F411106C6F1
:102B500022C426C25C45C04735CC93048401268537
:102B6000EFD01FA197E701009387C7909C43B5E77B
:102B7000930444002685EFD0BF9F97E70100938719
:102B8000279158549C4363F6E70097E7010023A17F
:102B9000E79093172700BA978A0717E501001305F6
:102BA000259EA6853E95EFD03F9897E70100938735
:102BB000A78F9C4358540145DC5763F8E7008547CD
:102BC00017E701002320F78C0545B24022449244C8
:102BD000410182807370043001A0A68517E50100D1
:102BE000130505A9EFD05F94C9B797E70100938754
:102BF00067889C4381E77370043001A0411106C6C9
:102C000022C426C2B70700804045CD8F1CC12DC409
:102C1000EFD01F96930444002685EFD07F9597E769
:102C200001009387E78658549C4363F6E70097E7D3
:102C3000010023AFE78493172700BA978A0717E5A7
:102C400001001305E5933E95A685EFD0FF8D97E72C
:102C50000100938767859C4358540145DC5763F80E
:102C6000E700854717E70100232EF7800545B240AE
:102C700022449244410182807370043001A011CD3E
:102C800097D701009387C77F984397E70100938701
:102C900067809C4318C15CC182807370043001A0BE
:102CA00055C1D1CD411106C622C42A8773700430A4
:102CB00097D801009388887D83A7080091CB97D788
:102CC00001009387677E94439C43FC428507FCC2C6
:102CD00017D301001303037C9C4103260300FD5618
:102CE0000144638FD70217DE0100130E6E790325AE
:102CF0000E000328070054436305A80005446371D0
:102D0000D6023308D6400544637CF80003250E0044
:102D1000918F03260300B6979CC108C350C301449A
:102D200083A7080081CB97D701009387E7779C435F
:102D3000FC4381EF2285B2402244410182807370BE
:102D4000043001A07370043001A0EF20B065DDB73E
:102D5000854717D701002327F772828019C168457C
:102D600082800145828011C16CC5828097D70100A5
:102D7000938787738843828097D701009387077171
:102D80009C43054589CB97D701009387A76E88435D
:102D9000133515000605828031CD011126CA97D45E
:102DA0000100938464709C4006CE22CC4AC84EC673
:102DB0005855DC576379F7021C4D63C707009C40E8
:102DC000D457A947958F1CCD93172700BA97584918
:102DD00017D901001309C97A8A07CA97630DF7004A
:102DE0009C40DC575CD5F2406244D2444249B2492F
:102DF000056182808280930945002A844E85EFD048
:102E00002FF79C4017D70100130787681843DC573A
:102E10005CD46376F70017D70100232BF766139570
:102E200027003E9562440A05F240D244CE854A9579
:102E3000B249424905616FD02FEF19CD411106C645
:102E400022C426C297D70100938707668043630791
:102E5000A4007370043001A0014582807C4881E7A2
:102E60007370043001A054543848FD177CC8638344
:102E7000E60099C70145B240224492444101828054
:102E8000930444002685EFD0AFEE3C4817D70100ED
:102E900013070760144329471D8F5CD418CC63F6D1
:102EA000F60017D701002325F75E5147B387E702E5
:102EB00017D501001305C56CA6853E95EFD0CFE66A
:102EC000054555BF7370043097D701009387075CA1
:102ED0009C4391CB97D701009387075D98439C4310
:102EE0007C4385077CC3828097D701009387075A6C
:102EF0009C438DC397D701009387075B9843784322
:102F000011CB984394437C43FD177CC3FC4299E367
:102F100073600430828097D701009387E75890430D
:102F200094439843A947D456084E958F1CCF82806E
:102F300097D7010093874757984309C79443F84AA6
:102F40000507F8CA8843828079714AD006D622D410
:102F500026D24ECE2A897370043097D40100938410
:102F6000E4529C4017D4010013040454BDE31C40F8
:102F7000BC4F89E71C400547F8CFD1E19C4081C791
:102F80001C40FC43F1EB737004309C408DEF1C40FF
:102F9000A84F11C5630409021C4023AC07041C4060
:102FA00023AE07049C4081C71C40FC438DEBB2500C
:102FB000225492540259F2494561828018403C4F94
:102FC000FD173CCFE9BF18401C407C4385077CC3FC
:102FD0007DBF18401C407C4385077CC349BF184017
:102FE00014407C43FD177CC3FC42F1F37360043052
:102FF000B250225492540259F249456182800840ED
:103000002EC61105EFD0CFD6B245FD576380F50629
:1030100097D701009387074883A9070018409C436E
:10302000AE992322370163ECF90497D70100938707
:10303000674788430C409105EFD08FD097D70100A8
:10304000938787439C4363F6F90097D7010023A534
:103050003743EFD0AFBB1DB7184014407C43FD177A
:103060007CC3FC428DF37360043031BF0C4017D534
:103070000100130565629105EFD00FCBD9BF97D73B
:1030800001009387E74188430C409105EFD04FCB77
:10309000C9B779714AD04ECE06D622D426D252CCA8
:1030A0002E89B2897370043097D401009384043E52
:1030B0009C4017D401001304243FF9EF18408947BE
:1030C000784F630CF7001C401345F5FFB84F798D1E
:1030D000A8CF1C400547F8CFADE69C4081C71C40F7
:1030E000FC43F5E3737004309C40B1E7638609004C
:1030F0001C40BC4F23A0F900184085470145784F7C
:10310000630BF7001C401349F9FF0545B84F3379AD
:10311000E90023AC27051C4023AE07049C4081C76F
:103120001C40FC43C1E3B250225492540259F2496C
:10313000624A4561828018401C407C4385077CC3FD
:1031400075B7084036C61105EFD08FC2B246FD579D
:103150006385F60897D701009387C73303AA070052
:1031600018409C43369A232247016363FA0897D795
:1031700001009387273388430C409105EFD04FBC63
:1031800097D701009387472F9C436370FA0697D720
:10319000010023A3472F91A818401C407C438507BA
:1031A0007CC329BF184014407C43FD177CC3FC42FC
:1031B000BDFB73600430B250225492540259F2495C
:1031C000624A45618280184014407C43FD177CC3ED
:1031D000FC4289FB7360043031B70C4017D5010005
:1031E0001305854B9105EFD02FB4EFD02FA2F5B585
:1031F00097D701009387C72A88430C409105EFD0E9
:103200002FB4E5B751C1411106C622C426C24AC037
:103210007370043097D40100938444279C40B9EB29
:1032200099C23C4D9CC2B2878946704D74CD2E87A1
:103230002A846386D70663FCF6048D456387B7004E
:1032400091456395B7006300D60C38CC8547630F72
:10325000F60405449C4081CB97D701009387C7248F
:103260009C43FC43A9E32285B24022449244024994
:103270004101828097D701009387072398439C439D
:103280007C4385077CC369BF7370043001A0854609
:10329000E39ED7FA3C4D33E7B70038CD45BF3C4DF0
:1032A00085073CCD65B7EF20F00F75BF13094400CB
:1032B0004A85EFD0EFAB17D701001307671D5C54A9
:1032C00018436376F70017D701002323F71C5147F3
:1032D000B387E70217D501001305852ACA853E95F5
:1032E000EFD08FA41C5481C77370043001A097D70E
:1032F00001009387671B9C435854DC57E3FBE7F4BA
:10330000EFD0CF90B9B70144B1B739CD011122CC7C
:1033100026CA4AC84EC652C456C206CEBA89368A92
:10332000B2842E892A84EFD04F9AAA8A63050A00B4
:103330003C4C2320FA00784C89477CCC6389F4020A
:1033400063F4970C8D466387D40091466396D4004E
:10335000630AF70A232C24058547631EF7061C54CD
:1033600099CB7370043001A07370043001A03C4C01
:1033700085073CCCD5B797D701009387A70F9C430F
:10338000ADEB930444002685EFD08F9E17D7010044
:10339000130707105C5418436376F70017D7010032
:1033A0002328F70E5147B387E70217D5010013050D
:1033B000251DA6853E95EFD02F9797D701009387BF
:1033C000A70E9C435854DC5763F7E7006385090058
:1033D000854723A0F90005445685EFD0AF8E22859E
:1033E000F2406244D2444249B249224A924A0561BB
:1033F00082809305840117D5010013056527EFD05E
:10340000AF9265BF0144C9BF8547E397F4F43C4CD4
:1034100033E92701232C240581B74DC1011122CCAA
:1034200026CA2A844AC806CE4EC6AE84EFD0EF899B
:103430008947744C7CCC3C4C05472A8985073CCC99
:103440006395E6061C5481C77370043001A097D7BA
:103450000100938727029C43ADE7930944004E8502
:10346000EFD00F9117D70100130787025C54184360
:103470006376F70017D70100232CF7005147B38775
:10348000E70217D501001305A50FCE853E95EFD0B5
:10349000AF8997D70100938727019C435854DC5785
:1034A00063F5E70099C085479CC06244F240D2446E
:1034B000B2494A85424905616FD0CF8073700430AC
:1034C00001A09305840117D501001305651AEFD0FB
:1034D000AF85C1B7AA8729C57370043017D701001B
:1034E0001307C7FA14439DE2F04F8946014563155F
:1034F000D60023AE070405451C4381CB97D70100B6
:10350000938787FA9843784315E3828097D6010022
:10351000938686F9904294427442850674C2E9B754
:1035200097D70100938747F89C437DB7984394430E
:103530007C43FD177CC3FC42E9FB7360043082804E
:103540005D71A6C2CAC052DC56DA5AD85ED686C6AB
:10355000A2C44EDE62D466D26AD017D90100130924
:10356000A9F517DB0100130B6BF497D401009384CA
:1035700024F497DA0100938AEAF3054AA54B8327DE
:103580000900984363010712DC4783A90700EFE0B5
:10359000EFF6EFE0AFF783270B002A8C6362F50AA2
:1035A00097D7010023A4A7F001466370351B88401C
:1035B000B3858941EFD0FFBDEFE05F99630105124C
:1035C0008840814601462C00EFD00FEC4DD9A24730
:1035D000E3C807FEC24983A7490189C7138549008B
:1035E000EFC01FF9EFE08FF283270B002A8C636D89
:1035F000F508A24717D70100232A87EBE3E2FBFC7B
:10360000B317FA0013F70721631A071613F7770C9D
:103610006318071E93F70702C5D74E85EF00F01118
:1036200045B7DC47C04783AC0700930944004E858B
:10363000EFC01FF45C50228582975C4C6384470B7B
:1036400083270900984371FF03A70A0097D601005A
:1036500023AE86E597D6010023AEF6E497D70100A6
:1036600023ACE7E4EFE09F8EA1BFDC47C04703AD8A
:103670000700930C44006685EFC09FEF5C502285E5
:1036800082975C4C6386470983270900984371FF42
:1036900003A70A0097D6010023AEF6E097D70100F2
:1036A00023ACE7E0B9B7EFE06FE5EFE02FE6832763
:1036B0000B002A8CE366F5F883A70A00884081494D
:1036C0009043B385894117D70100232187DF133643
:1036D0001600EFD01FACEFE07F87E31305EEEFC0DD
:1036E000FFD2F9BD1C4CCE85E69763E9FC049C40F3
:1036F00089CF02CA66CC22CEEFF00FE8884081461F
:1037000001464C08EFD02F8805FD7370043001A0EE
:103710001C4CE685EA97636CFD049C4089CF02CA85
:103720006ACC22CEEFF04FE58840814601464C0836
:10373000EFD06F8531F97370043001A003250900C3
:103740005CC000C8EFC0DFDFE5BDEFE03F8083274E
:103750000900DC47C047930C44006685EFC05FE179
:103760005C4C638F47035C502285829791BD032593
:1037700009005CC000C8EFC0BFDC39B7B24723AC5A
:10378000F900A5CFE29723A2F90023A83901938578
:103790004900636FFC0403A50A00EFC07FDA0DB592
:1037A0001C4C00C83387F90058C0636DEC02330C21
:1037B0003C416363FC029C4089CF02CA4ECC22CEBE
:1037C000EFF08FDB8840814601464C08EFC0BFFB1D
:1037D00059F97370043001A003A50A00E685EFC013
:1037E0003FD651B703250900E685EFC07FD5A5BFB9
:1037F00003250900EFC0DFD4E1B37370043001A0EA
:10380000B24783A6890123A839013387D70023A2B1
:10381000E9006364EC04B307FC4063EBD70483A7BF
:1038200049024E85829783A7C901E39B47D983A6A6
:103830008901B2479840B69711CF02CA3ECC4ECE0E
:10384000EFF08FD38840814601464C08EFC0BFF3AC
:10385000E31805D67370043001A06374FC00E370B4
:10386000F7FC0325090093854900EFC07FCD89BB94
:1038700003A50A0093854900EFC09FCC91B3411185
:1038800022C406C626C24AC017D40100130444C28B
:10389000EFF04FE31C4095CBEFF00FE51C409DC3CC
:1038A000814801488147094781461306004097D562
:1038B00001009385A5B0170500001305A5C8EFD03A
:1038C0007F9A39E97370043001A017D901001309F8
:1038D000E9DD4A85EFC0BFC397D40100938444DE7D
:1038E0002685EFC0DFC20146B145114597D70100DB
:1038F00023A427BD97D7010023AE97BAEFC01FDCE2
:1039000017D701002326A7BA11CD97D501009385BB
:1039100065AAEFD0CFFC49B7B24022449244024995
:10392000410182807370043001A0A5C9797156CA23
:10393000AA8A1305C00222D426D24AD04ECE52CC37
:1039400006D65AC85EC63A89B689328AAE84E9215B
:103950002A8405C9EFF00FD797D70100938747B5A1
:103960009C439DCFEFF04FD8130544002320540112
:1039700004CC232E44012320340323222403EFC04C
:103980005FBA2285B250225492540259F249624AD7
:10399000D24A424BB24B456182807370043001A021
:1039A00097DB0100938B8BD05E85EFC05FB617DB92
:1039B0000100130BEBD05A85EFC07FB50146B1452E
:1039C000114597D7010023A977AF97D7010023A30B
:1039D00067AFEFC0BFCE17D70100232BA7AC01C93B
:1039E00097D501009385059DEFD06FEFA5BF73704C
:1039F000043001A039C5011122CC06CE26CA17D445
:103A000001001304E4AA832804002A880145638581
:103A10000802BA842EC2368732C442C6954663C5B0
:103A2000B602EFF06FB58947630BF5020840814697
:103A300001464C00EFC03FD5F2406244D2440561DC
:103A400082807370043001A04C0081463A8646851E
:103A5000EFD0AF88F2406244D244056182800840D2
:103A6000814626864C00EFC01FD2F9B719C1084124
:103A700082807370043001A001E57370043001A0EE
:103A8000411106C622C42A84EFF0CFC3484833341C
:103A9000A000EFF06FC52285B24022444101828030
:103AA00001E57370043001A0411122C42A8406C6C6
:103AB000EFF04FC10050EFF02FC3B24022852244F7
:103AC0004101828001E57370043001A0411122C4DC
:103AD00026C22E84AA8406C6EFF0CFBE80D0224430
:103AE000B240924441016FF02FC04111714522C490
:103AF00006C61D262A8411C5232005001105EFC026
:103B00001FA12285B24022444101828001CDB70726
:103B100000FFED8F81C77370043001A099E57370C9
:103B2000043001A07370043001A0011122CC4AC8F6
:103B30004EC652C456C206CE26CABA893689B28A41
:103B40002E842A8AEFF04FA311E563850900737074
:103B5000043001A0EFE08F9A83240A00B377940029
:103B60006316090295C763870A009347F4FFE58F40
:103B70002320FA00EFE08FBDF240624426854249DF
:103B8000D244B249224A924A05618280E30DF4FC94
:103B9000E38209FEB3355001E20563050900B7076A
:103BA0000004DD8D4E86C18D13054A00EFE0FFE66F
:103BB000EFE0CFB919E1EFC07F85EFF0CFB59317F4
:103BC0006500AA8963D80700B7040001FD14B3F4A7
:103BD00099005DB7EFF00FAF83290A00B377340186
:103BE000631E090089CB63880A009347F4FFB3F78B
:103BF00037012320FA00EFF02FAFF9B7E31DF4FEF1
:103C0000DDB701C9B70700FFED8F99C773700430A6
:103C100001A07370043001A0411122C42A8406C699
:103C200026C24AC02E89EFF0EFA904409345F9FF60
:103C3000B3F795001CC0EFF02FABB24022442685AD
:103C40000249924441018280411122C42A8406C65D
:103C5000EFC0BF870040EFC0FF86B24022852244FC
:103C60004101828009C9370700FFB3F7E50099C712
:103C70007370043001A07370043001A06F10507491
:103C8000B70700FFF18F81C77370043001A001E610
:103C90007370043001A0011122CC4AC84EC652C430
:103CA00006CE26CA3689AE892A8A3284EFF0CF8CB6
:103CB00021E1630509007370043001A0EFE00F8477
:103CC00083240A00CE855285B3E49900613FB3771F
:103CD00094006307F40683240A00EFE02FA7F24064
:103CE000624426854249D244B249224A0561828013
:103CF000EFE0CF8083240A00CE855285B3E43401FF
:103D00009537B3F78400638D8702E30609FCB70596
:103D100000054A86C18D13054A00EFE01FD0EFE091
:103D2000EFA219E1EFC08FEEEFF0EF9E9317650061
:103D3000AA8463DF0700B7070001FD17FD8C45B7B4
:103D400083270A001344F4FFE18F2320FA0071B7A0
:103D5000EFF04F9783240A00B377940063978700AE
:103D60009347F4FFE58F2320FA00EFF0EF97E1B7D8
:103D7000411122C406C62A8426C2EFD03FF85C4017
:103D800085C308489304C4006316950015A008482D
:103D900063009502B7050002EFE03FE55C40E5FBFC
:103DA0002285612A2244B240924441016FE00F9A79
:103DB0007370043001A009C9370700FFB3F7E500AD
:103DC00099C77370043001A07370043001A06F10A4
:103DD000305F01C9B70700FFED8F99C773700430DA
:103DE00001A07370043001A0411122C426C206C68E
:103DF0002A84AE84EFF00F8D184093C7F4FFF98F3B
:103E00001CC02244B240924441016FF0EF8D19C1B1
:103E1000084D828001458280411122C406C62A8451
:103E2000EFD0DFED97C70100938747699C43A1EB73
:103E3000E56717D701001307278AF11797C6010016
:103E400023A4E66817C70100232EF76617D70100E1
:103E50002326F78897C701009387876617D7010045
:103E6000232CF786854717C701002321076617C74C
:103E700001002327076417C701002321F76419E80D
:103E8000EFE0CF8CEF10E00501442285B2402244E0
:103E9000410182801305840093773500C1EFE56707
:103EA0001307F5FFE917E3EDE7FC97C601009386DA
:103EB000A6619C4229A0984311C7BE86BA87D84301
:103EC000E36BA7FE17C701001307875FE38AE7FAD2
:103ED000984341461384870098C2D843B306A7404D
:103EE0006378D6023388A7002322D800C8C383256D
:103EF000480097C601009386265D11A0BA869842B5
:103F00005043E36DB6FE2320E80023A00601D8430A
:103F100097C701009387475D9C43998F17C701009E
:103F20002324F75CEFE08F8231DC2285B24022440B
:103F300041018280719911059DB729C9411122C49F
:103F400006C62A84EFD09FDB930584FF0326C4FFB7
:103F500017C701001307475711A03E871C43D443DE
:103F6000E3EDC6FE232CF4FE0CC397C70100938734
:103F7000A75798438327C4FF2244B240BA9717C774
:103F800001002323F75641016FD05FFC828097C761
:103F90000100938767558843828082803367B5002C
:103FA0000D8BAA871DE79308D6FFAA982A87AE86AD
:103FB0006371150303A8060011079106232E07FF5E
:103FC000E36A17FF9347F5FFC697F19B9107BE95EC
:103FD000AA972A9663F3C70A938645001388470079
:103FE000B3B6D70033B8050133E7F50093C6160022
:103FF000134818000D8BB3E6060113371700758FB1
:10400000330EF6409386170029CF1337AE0031EBFD
:1040100013532E002E88BE8601478328080005070B
:10402000110823A016019106E36967FE1377CEFFFE
:10403000BA95BA976302EE0483C60500138717008A
:104040002380D700637AC70283C615001387270031
:10405000A380D7006372C70203C725002381E7004E
:104060008280B307F640AE97850503C7F5FF850646
:10407000238FE6FEE39AF5FE82808280B367C50057
:104080008D8BB308C500E9C36371150FB307A0405A
:104090008D8B13873700954693F5F50F13081500A0
:1040A0003383A8407D166373D70015476363E60C1E
:1040B000D5CF2300B5000547638DE700A300B50009
:1040C0000D47130825006396E70013083500230108
:1040D000B500139685004D8E13970501518F33035C
:1040E000F34093968501D98E13562300AA97014772
:1040F00094C305079107E36DC7FE1377C3FFB307AA
:10410000E8006307E3062380B70013871700637C8A
:104110001703A380B7001387270063761703238153
:10412000B7001387370063701703A381B7001387A5
:104130004700637A17012382B7001387570063741F
:104140001701A382B700828093F5F50F13978500BE
:10415000D98D139705014D8FE37715FFAA87910736
:1041600023AEE7FEE3ED17FF828082802A8895B7B1
:104170008280AA8749BF834705002A8799C705051A
:1041800083470500EDFF198D82800145828005057A
:104190008347F5FF850503C7F5FF91C7E389E7FE70
:1041A0003385E74082808147E5BFAA87850503C73D
:1041B000F5FF8507A38FE7FE75FB82808346050028
:1041C000930700026397F600050583460500E38D1B
:1041D000F6FE938756FD93F7D70F85C7AA878145CB
:1041E00085CE01458507138606FD1317250083C676
:1041F00007003A9506053295F5F699C13305A040BA
:104200008280938536FD8346150093B5150093078C
:104210001500E1FA0145D5B7014582809C41238014
:10422000A7009C4185079CC1828097C601009386A8
:10423000262A9C42175703001307C74C1386170002
:10424000BA972380A70097C5010023A3C528A947D3
:104250006308F500930700046305F60001458280BA
:1042600075DE370610F005078347F7FF2320F6F0C9
:104270009C42FD1797C5010023ACF524EDF70145DD
:1042800082804D712322911423202115232A51135A
:10429000232481132326111423248114232E311364
:1042A000232C4113232861132326711323229113F6
:1042B0002320A113232EB111AA842E8932C6130CF8
:1042C0005002A54A8347090063808703B9CB804029
:1042D00011A0A1CB2300F40080400509050480C093
:1042E00083470900E39787FF0346190093081900E5
:1042F000C686130D0002FD597D5A0148130550056D
:104300009307D6FD93F7F70F138916006363F52A19
:1043100017C70100130707CF8A07BA979C43BA97BC
:1043200082878320C1140324811483244114032928
:1043300001148329C113032A8113832A4113032BF8
:104340000113832BC112032C8112832C4112032DE4
:104350000112832DC11171618280A14C02C4854775
:1043600063D50715B2478040938B770093F68BFF98
:1043700003AB060083A94600938786003EC6668687
:1043800081465A85CE85EF1060462AC881476385ED
:104390003723930D4101854B668681465A85CE852C
:1043A000EF10E00E814666862A8BAE89EF1000443E
:1043B000A24723A0AD0093861B00910D63843701B3
:1043C000B68BD9BFE37E9BFF63DD4601A2872380C6
:1043D000A70180407D1A930714009CC03E84E3C867
:1043E00046FF93962B001C08BE9631A8938777054D
:1043F0002300F4008040FD1B93871B00050480C050
:10440000F116E351F0EC9C42E3E2FAFE93870703D6
:10441000C5B79C409306000332472380D7009C40D9
:1044200093064700C14C1386170090C013068007FF
:10443000A380C700804002C4BA87050480C003ABD4
:104440000700814936C625BFB24783AC0700938B6E
:10445000470063840C1C635F40199307D002631903
:10446000FD1683C70C0085C363DC09189440850CD6
:104470007D1A2380F6008040050480C083C70C00AD
:10448000E5F7635D40018040930700022300F400DC
:1044900080407D1A050480C0E31A0AFE5EC61DB581
:1044A00002C48547A94CE3CF07EBB247804093860F
:1044B000470071B703C61600CA8699B59C4093069B
:1044C00050022380D7008040050480C0E5BBC14C6A
:1044D00002C471B5B24703C61600CA8683A9070095
:1044E00091073EC6E35E0AE04E8AFD5911BD03C640
:1044F0001600130DD002CA8621B59347FAFFFD8737
:1045000003C61600337AFA00CA86DDBB03C616005E
:10451000130D0003CA86EDB383C51600930906FD8B
:10452000CA86938705FD2E86E3EEFAFA9397290053
:10453000BE9985068609AE9983C50600938909FD53
:10454000938705FD2E86E3F3FAFE69BF32479C4050
:10455000144311073AC62380D7008040050480C069
:1045600095B3854763D3070BB24793867700E19AEB
:10457000938786003EC683A946009C4263DC090AF5
:1045800094401306D002B307F0402380C600804059
:10459000B336F000B3093041050480C03E8BB389C7
:1045A000D940A94C02C4E1BB03C616000508CA865F
:1045B00081BB9C40468921B7E37D9BDD8547814BCC
:1045C0008546E3C547E131BD97CC0100938C8CDF74
:1045D000CE856685EF009031330AAA40635C4001C6
:1045E00080402300A40180407D1A050480C0E31AA6
:1045F0000AFE014A83C70C00E38207EAE3C809E622
:10460000FD197D57E394E9E6ADBDB24793864700B7
:104610009C4336C693D9F74195B76356400193073B
:10462000D002E313FDFA97CC0100938CACD9930729
:1046300080021DBD3E8BA94C02C4804089B34D71E0
:10464000232E3113B70900409387F9FF23248114E7
:1046500023229114232C4113232A511323261114AE
:10466000232021152328611323267113232481136A
:10467000232291132320A113232EB1112A8A2EC4A1
:1046800017C401001304C4E4975A0300938A8A07ED
:1046900097C40100938484AC3EC69305500229451B
:1046A00013080004B70610F083470A006386B704B6
:1046B000C1C71840050A13061700569797C801008E
:1046C00023A8C8E02300F7006382A706E31E06FDC7
:1046D000175703001307070305078347F7FF23A0B6
:1046E000F6F01C40FD1717C601002323F6DEEDF798
:1046F00083470A00E39EB7FA83461A0013051A009F
:104700002A87930B00027D5B7D5C01489305500571
:10471000A5489387D6FD93F7F70F130A170063E7B1
:10472000F5348A07A6979C43A697828717570300FC
:10473000130747FD55F28DBF8320C1140324811454
:1047400083244114032901148329C113032A8113EB
:10475000832A4113032B0113832BC112032C8112D3
:10476000832C4112032D0112832DC11171618280AE
:10477000A14C014D854763DB0719A2479D07E19BCB
:1047800083AD070003AB4700138787003AC46686F2
:1047900081466E85DA85EF1060052AC863066D359F
:1047A000130941018549668681466E85DA85EF00E9
:1047B000104E66868146AA8D2E8BEF102003232093
:1047C000A90085091109E3106DFFE3FE9DFD1306A5
:1047D0000004B70610F063D189031C40138717004B
:1047E000D69797C5010023A5E5CE23807701630CFA
:1047F000C7047D1CE3C389FFB2476800A548B386A0
:10480000F9008A061C08BE962948130300043706DF
:1048100010F0E384A6E89C429305000363F4F800DB
:10482000930570051840AE9793051700569717CE5D
:104830000100232FBEC82300F7006380072B638C81
:104840006526F116F9B7175703001307A7EB0507FD
:104850008347F7FF23A0F6F01C40FD1797C5010022
:1048600023A8F5C6EDF77D1C71B71C4013060004A4
:104870001387170097C5010023ACE5C4B386FA007F
:10488000930500032380B600630FC73C890797C6D2
:10489000010023AFF6C25697930680072300D70086
:1048A00017570300130707E6B70610F0639EC7000B
:1048B00005078347F7FF23A0F6F01C40FD1717C636
:1048C00001002327F6C0EDF7A247C14C014D910727
:1048D0002247014B832D07003EC455BDA24783AC40
:1048E000070013894700638E0C3A635480219307B5
:1048F000D002639EFB2E03C70C00BA85631007200D
:1049000025AC8547A94C014DE3C907E7A2479107AC
:10491000C1B7A24783461700528703AB0700910730
:104920003EC4E3580CDE5A8C7D5BE5B3834617002A
:10493000930BD0025287F1BB9347FCFFFD87834660
:104940001700337CFC005287E9B383461700930BB2
:10495000000352877DBB03461700138B06FD528769
:10496000930706FDB286E3EEF8FA93172B00DA9769
:1049700005078607B29703460700138B07FD9307C9
:1049800006FDB286E3F3F8FE69BFA2451C40294646
:10499000984193861700D69717C50100232AD5B2F0
:1049A0002380E700138945006300C72A93070004AA
:1049B0006387F6204AC4D5B1854763DE0729A2473D
:1049C00013877700619B930787003EC4032B470042
:1049D0001C43635A0B30184013060004930617005B
:1049E00097C5010023A6D5AE56979305D0022300A4
:1049F000B7006387C62CB307F0403337F000330BA2
:104A00006041BE8D330BEB40A94C014D49B3834649
:104A1000170005085287F5B9834617005287D5B9A4
:104A20001C40930600041387170017C601002321BA
:104A3000E6AAD697130650022380C700E31FD7C407
:104A400017570300130707CCB70610F00507834775
:104A5000F7FF23A0F6F01C40FD1717C6010023291D
:104A6000F6A6EDF71DB9C14C014D29B31C409306C4
:104A700000042A8A1387170017C60100232AE6A418
:104A8000D697130650022380C700E318D7C01757E4
:104A90000300130727C7B70610F005078347F7FF82
:104AA00023A0F6F01C40FD1717C601002322F6A232
:104AB000EDF72A8ADDB6175703001307A7C40507C9
:104AC0008347F7FF2320F6F01C40FD1797C5010030
:104AD00023A0F5A0EDF7F1162DBB17570300130720
:104AE00067C2F1FDF11635B3E3FC9DCB8549C5B135
:104AF000014C03C70C00BA85E30E07EAFD582945AF
:104B000013080004B70610F063570B0A1C40138605
:104B10001700D69717C30100232CC39A2380E70000
:104B20006384A50663040609850C03C70C007D1C7D
:104B3000BA8579FBE35080E91C4093050002130617
:104B40000004B70610F021A07D1CE3050CE61387D6
:104B50001700D6972380B70017C50100232AE596D2
:104B6000BA87E313C7FE175703001307A7B9050752
:104B70008347F7FF23A0F6F01C40FD1717C501007F
:104B80002328F594EDF7C9B717570300130787B724
:104B900041DE05078347F7FF23A0F6F01C40FD1711
:104BA00017C601002326F692EDF7BDBF1757030085
:104BB000130747B5F9BF7D1BE31A1BF5A5BF1757B0
:104BC0000300130727B4B70610F005078347F7FF64
:104BD00023A0F6F01C40FD1717C60100232AF68E0D
:104BE000EDF74AC45DBC97BC0100938CAC7DDA85BF
:104BF0006685ED29330CAC40E35D80EF1C40130665
:104C00000004B70610F021A07D1CE3030CEE13870F
:104C10001700D6972380770197C5010023AAE58A5C
:104C2000BA87E313C7FE175703001307A7AD05079D
:104C30008347F7FF23A0F6F01C40FD1797C501003E
:104C400023A8F588EDF7C9B717570300130787ABFB
:104C5000BDFA4AC499B4A247138747009C433AC49B
:104C600013DBF741BDB3175703001307A7A9B70616
:104C700010F005078347F7FF23A0F6F01C40FD174F
:104C800017C601002326F684EDF7854717C70100F4
:104C90002320F78493078007175703002304F7A600
:104CA00025B1635680019307D002E39EFBF297BCC7
:104CB0000100938C2C7113078002930580023DBD87
:104CC00097560300938606A4370610F0850603C79F
:104CD000F6FF2320E6F018407D1797B5010023A9C1
:104CE000E57E6DF709BBBE8DA94C014D4DB4B707EC
:104CF00010F023A0A7F201A03971130341022ED2B4
:104D00009A8506CE32D436D63AD83EDA42DC46DE32
:104D10001AC63532F2400145216182805D7113036C
:104D2000810322D42AC632DC2A841A86680006D679
:104D3000BEC236DEBAC0C2C4C6C61ACEEFF06FD449
:104D4000B247238007003245B250018D2254616181
:104D50008280B70710F083A647F403A607F403A7E1
:104D600047F4E31AD7FE8566938606FAB29633B601
:104D7000C600B305E60023A4D7F423A6B7F48280C7
:104D8000B70710F003A747F403A607F483A647F478
:104D9000E31AD7FE8566938606FAB29633B6C60046
:104DA00023A4D7F4B305E60023A6B7F493070008BD
:104DB00073A04730828085AC411122C406C697B7E4
:104DC00001009387677117B401001304A47098431E
:104DD0001C401306F07C930647069387470697B559
:104DE000010023ABD56E97B5010023A5F56E634690
:104DF000D600B2402244410182801307478997B709
:104E0000010023ABE76CDD2A8547631FF5001840DE
:104E100085679387F7760145E3DDE7FCC93D2244CA
:104E2000B24041016FC09FEC17B501001305055A50
:104E3000E13509456D3D2244B24041016FC01FEB91
:104E400017B501001305C55A45BD17B50100130577
:104E5000A55A5DB5411122C426C206C6856417B4A1
:104E600001001304E459938784380100FD17F5FF0E
:104E700022855935CDBF4111014506C622C4352AC8
:104E800017070000130767F38146054693052003C3
:104E900017B5010013054557EFE03FA92A84EFC07D
:104EA000FFE62A8622852244B24001478146854595
:104EB00041016FE03FB4411106C689220547814791
:104EC0006316E500B2403E854101828017B50100BE
:104ED0001305C54FEFF05FE2B24089473E854101BF
:104EE00082807370043001A082807370043001A04E
:104EF000797101469145054506D622D426D24AD07D
:104F00004ECE52CCEFB08FFB55C5AA84054417BADC
:104F10000100130A2A5DA9491149894601462C005E
:104F200026854EC4EFB03F86814601462C0026857B
:104F300002C4EFB07FD5A24702C6D91793B71700B6
:104F4000B307F0407D8C894601466C002685EFB0A2
:104F50009F83854601462C002685EFB0FFD2A247ED
:104F600032472685998F93B71700B307F0407D8CA1
:104F7000EFC06F87B2477D151335150085073305E0
:104F8000A0403EC6698CE370F9FC814601462C00C6
:104F90002685EFB07FCF2685EFC0EF8411E935DCA1
:104FA00083270A00850717B70100232DF752B5B7ED
:104FB0000144A5B77370043001A0411122C4014619
:104FC0002A849145054506C6EFB04FEF228722445B
:104FD000B24097B7010023A5A750814801488147F7
:104FE00081461306004097B50100938525431705B8
:104FF0000000130525F041016FC0CFA697B701004F
:105000009387074F9843854701456319F70097B782
:1050100001009387274D88433335A00097B70100DF
:1050200023A2074C828079714ECE97B901009389F3
:10503000294B03A5090026D24AD0D144294906D6D6
:1050400022D44AC226C43DC917B40100130404493E
:105050001C4005476387E7069DCF0947639EE7002D
:1050600001466C00EFB03FE8B247638197061C40F1
:1050700017B70100232E074685070947637DF7040C
:10508000B250225497B7010023AA07449254025900
:10509000F24945618280894601464C00EFB0FFA38A
:1050A00003A509006C00EFB0DFEDB2476380270372
:1050B00097B7010023AE07421C407DBF73700430D8
:1050C00001A0894601462C00EFB03FA11C400947D2
:1050D0008507E367F7FAB250225417B70100232F70
:1050E000F73E92540259F24945618280AA95AA87F7
:1050F0006385B70003C7070001E73385A7408280B7
:105100008507FDB7814863DA05003305A040B33752
:10511000A000B305B0409D8DFD5863D9060033064D
:10512000C040B337C000B306D0409D8E328836836E
:10513000AA872E87639F061C97B601009386861761
:1051400063F1C50C416E6377C60B130EF00F6373EA
:10515000CE002143335E6600F29603CE06001A9E0F
:10516000130300023303C341630C0300B3956500CE
:10517000335EC501331866003367BE00B3176500A0
:10518000135E0801B355C70313150801418193D677
:1051900007013376C703B305B5024206D18E63F823
:1051A000B600C29663E5060163F3B600C2968D8E23
:1051B00033F7C603C207C183B3D6C603B306D5020D
:1051C00013150701C98F63F8D700C29763E507017C
:1051D00063F3D700C297958F33D567008145638A03
:1051E0000800B307A0403337F000B305B0403E8558
:1051F000998D8280370E00014143E36DC6F561430E
:1052000091BF01E605483358680241676373E808B7
:105210001307F00F63730701214333576800BA96F1
:1052200003C606001A96130300023303C340631932
:105230000306B38505419356080113150801418102
:1052400013D6070133F7D502B3D5D5024207518FE4
:10525000B305B5026378B7004297636507016373CE
:10526000B7004297B305B74033F7D502C207C183F1
:10527000B3D5D502B305B50213150701C98F63F87D
:10528000B700C29763E5070163F3B700C2978D8F3C
:10529000A1B7370700014143E361E8F86143B5BFB7
:1052A0003318680033DEC500935E08013356C5002D
:1052B000B31765003355DE03B39565004D8E931526
:1052C0000801C181935606013377DE033385A502B9
:1052D0004207558F6378A7004297636507016373A0
:1052E000A7004297B306A74033F7D6034206418290
:1052F000B3D6D6034207B386D502B365C70063F8B9
:10530000D500C29563E5050163F3D500C295958D7F
:105310001DB7E3E6D5EC416863F50605930EF00F83
:1053200033B8DE000E0833DE060117B301001303A5
:1053300063F87293834E0300130E0002C29E330E75
:10534000DE4163170E0263E4B6006369C500B3076C
:10535000C540958D3335F5003387A5403E85BA8528
:10536000BDBD370300014148E3EF66FA614865BF00
:105370003357D601B396C601D98EB357D50133D76B
:10538000D501B395C501CD8F93D506013373B7020F
:10539000139F0601135F0F0113D807013316C601CF
:1053A0003315C5013357B702420333680301B30F06
:1053B000EF023A83637CF80136981303F7FF6367C3
:1053C000D8006375F8011303E7FF36983308F841F6
:1053D000B37FB8023358B802C20FB3050F03139F4F
:1053E0000701135F0F0133EFEF014287637CBF00BA
:1053F000369F1307F8FF6367DF006375BF0013076D
:10540000E8FF369F4203C16F3363E3009387FFFFDA
:1054100013580601330FBF40B375F3001353030154
:10542000F18F3387F502B307F302B3850503330326
:105430000303BE95135807012E986373F8007E93FB
:10544000C167FD17935508013378F80042087D8F36
:105450009A9542976366BF00631BBF006379E500BE
:105460003306C7403337C700958D998D3287330790
:10547000E5403335E500B305BF40898DB397D501CD
:105480003357C70133E5E700B3D5C50189BBAE8704
:10549000328836872A836396062097B8010093885E
:1054A00068E163FEC50A41676374E60A1307F00FFB
:1054B0003337C7000E07B356E600B69883C6080018
:1054C000369793060002998E99CAB397D70033573F
:1054D000E5003318D600B365F7003313D500135534
:1054E0000801B3D7A50213160801418293560301A0
:1054F00033F7A502B305F6024207D98E3E8763FC57
:10550000B600C2961387F7FF63E7060163F5B6009E
:105510001387E7FFC2968D8EB3F7A602420313539B
:105520000301B3D6A602C20733E36700B305D60270
:105530003685637BB30042931385F6FF63660301F0
:105540006374B3001385E6FF4207498F81454DA878
:10555000B70600014147E360D6F66147A9BF01E6FF
:10556000854633D8C602C166637ED8089306F00F1D
:1055700063F306012147B356E800B69883C60800D6
:10558000BA9613070002158F49E7B387074185458F
:10559000135608019318080193D808019356030184
:1055A00033F7C702B3D7C7024207D98E3385F80253
:1055B0003E8763FCA600C2961387F7FF63E70601E8
:1055C00063F5A6001387E7FFC296898EB3F7C6027C
:1055D000420313530301B3D6C602C20733E3670085
:1055E000B388D8023685637B130142931385F6FF97
:1055F00063660301637413011385E6FF4207498F55
:105600003A858280B70600014147E366D8F66147D4
:105610009DB73318E800B3D5D7003313E500B35670
:10562000D50013550801B397E70033F7A502B3E897
:10563000F60093170801C18313D60801B3D5A5025C
:105640004207518FB386B7022E86637CD7004297FC
:105650001386F5FF636707016375D7001386E5FFBF
:105660004297B306D74033F7A602C20893D8080181
:10567000B3D6A6024207B385D702B36717013687B0
:1056800063FCB700C2971387F6FF63E7070163F572
:10569000B7001387E6FFC2978D8F93150601D98D4A
:1056A000C5BD63E2D514416763FEE6021308F00F3F
:1056B0003337D8000E0733D8E60097B5010093853D
:1056C00065BFC29503C80500930500023A98B385EB
:1056D000054185E10547E3E5F6F23335C50013479B
:1056E000150039BFB70500014147E3E6B6FC614745
:1056F000D9B733570601B396B600D98E93DE0601AB
:1057000033D70701B378D703B397B70033580501F0
:105710003363F80093970601C183135803013316CE
:10572000B6003357D703C20833E80801338FE702C6
:105730003A8E637CE8013698130EF7FF6367D80052
:105740006375E801130EE7FF36983308E841B37834
:10575000D8033358D803C208B38E07039317030145
:10576000C183B3E7F800428763FCD701B6971307FC
:10577000F8FF63E7D70063F5D7011307E8FFB69793
:10578000420EB387D741C16E3367EE001388FEFF28
:105790003373070193580701337806014182330EB2
:1057A00003033388080393560E013303C302429365
:1057B0009A96B388C80263F30601F69813D60601D9
:1057C000B29863E01703E39317D9C167FD17FD8E05
:1057D000C206337EFE003315B500F2968145E371B3
:1057E000D5E27D17A5B38145014719BDB28836873B
:1057F000AA872E886398061C97B60100938686AB0D
:1058000063F8C50A4163637E66081303F00F637390
:10581000C30021473353E6009A9603CE06001303D4
:1058200000023A9E3303C341630C0300B395650045
:10583000335EC501B31866003368BE00B317650058
:1058400013D608013377C80213950801418193D616
:1058500007013358C8024207D98E3308050363F89D
:105860000601C69663E5160163F30601C696B38684
:10587000064133F7C602C207C183B3D6C602B306D8
:10588000D50213150701C98F63F8D700C69763E5E2
:10589000170163F3D700C697958F33D5670081450D
:1058A0008280370300014147E36666F661479DB792
:1058B00001E60546B3581603416663F3C8081306AC
:1058C000F00F63731601214733D6E800B29603CE7A
:1058D0000600130300023A9E3303C3416319030613
:1058E000B385154113D7080113950801418113D6DB
:1058F0000701B3F6E502B3D5E502C206D18EB305C2
:10590000B50263F8B600C69663E5160163F3B60008
:10591000C696B385B640B3F6E502C207C183B3D5D8
:10592000E502B305B50213950601C98F63F8B70008
:10593000C69763E5170163F3B700C6978D8FB1BFB4
:10594000370600014147E3E1C8F86147B5BFB398A6
:10595000680033D7C501B3176500335EC50113D5A1
:105960000801B376A702B3956500336EBE00939528
:105970000801C18113560E013357A702C206D18E0A
:105980003387E50263F8E600C69663E5160163F324
:10599000E600C6963386E640B376A602420E135E54
:1059A0000E013356A602C2063386C502B3E5C60110
:1059B00063F8C500C69563E5150163F3C500C69598
:1059C000918D0DB7E3EED5EC416763F5E604930ED8
:1059D000F00F33B7DE000E0733D3E60097B80100AF
:1059E0009388488D9A9883CE0800130E0002BA9EC1
:1059F000330EDE4163170E0263E4B6006369C5002F
:105A0000B307C540958D3335F5003388A5403E85F5
:105A1000C28579B5B70800014147E3EF16FB61473E
:105A200065BF3357D601B396C601D98EB357D5019A
:105A300033D7D501B395C501CD8F93D50601337307
:105A4000B702139F0601135F0F0193D807013316A6
:105A5000C6013315C5013357B7024203B3681301BA
:105A60003308EF023A8363FC0801B6981303F7FF8B
:105A700063E7D80063F508011303E7FFB698B3881E
:105A80000841B3FFB802B3D8B802C20FB3051F0371
:105A9000139F0701135F0F0133EFEF014687637C0C
:105AA000BF00369F1387F8FF6367DF006375BF0091
:105AB0001387E8FF369F4203C1683363E30093878F
:105AC000F8FF13580601330FBF40B375F3001353AB
:105AD0000301F18F3387F502B307F302B3850503A2
:105AE00033030303BE95135807012E986373F80020
:105AF0004693C167FD17935508013378F8004208B3
:105B00007D8F9A9542976366BF00631BBF006379E0
:105B1000E5003306C7403337C700958D998D32872E
:105B20003307E5403335E500B305BF40898DB397B2
:105B3000D5013357C70133E5E700B3D5C5018DB3B0
:105B400097B7010093874796944317B7010013074F
:105B500067941843C8C2637BE50017B701001307B9
:105B6000279408438C4391056FA09F9D411122C447
:105B700006C617B701001307E7922A8408438C432F
:105B80009105EFA0FF9B97B701009387E78E9C4399
:105B90006376F40097B7010023A0878EB2402244B9
:105BA0004101828097B701009387079098439443FF
:105BB0007C43FD177CC3FC4299E373600430828010
:105BC000011122CC26CA2A84AE844AC84EC652C4C9
:105BD00056C206CEEFC08F921C4003290401B709BC
:105BE0000001B3E59700930AC4000CC08144FD197D
:105BF000370A00021840638C2A03032609004A85ED
:105C0000B3654701B376360193175600758F0329A4
:105C1000490063C4070001E7F1BFE39DE6FC931769
:105C2000760063D30700D58CEFC03FFCE1B793C487
:105C3000F4FFF98C04C0EFC06FB10840F240624439
:105C4000D2444249B249224A924A056182804111B6
:105C500006C622C4EFF02FA217F7FFFF130707169F
:105C6000814605469305400617A501001305457AB0
:105C7000EFD0BFCB19C92A84EFC04F892A860147CC
:105C8000814685452285EFD0FFD6EFB0BFE1B24017
:085C900022440145410182801C
:02000004800278
:10000000B444FEFFB245FEFFBC44FEFFB245FEFF16
:10001000B245FEFFB245FEFFB245FEFFD444FEFFEF
:10002000B245FEFFB245FEFFEE44FEFFFA44FEFF7E
:10003000B245FEFF0C45FEFF1845FEFF1845FEFFCA
:100040001845FEFF1845FEFF1845FEFF1845FEFF48
:100050001845FEFF1845FEFF1845FEFFB245FEFF9E
:10006000B245FEFFB245FEFFB245FEFFB245FEFFC0
:10007000B245FEFFB245FEFFB245FEFFB245FEFFB0
:10008000B245FEFFB245FEFFB245FEFFB245FEFFA0
:10009000B245FEFFB245FEFFB245FEFFB245FEFF90
:1000A000B245FEFFB245FEFFB245FEFFB245FEFF80
:1000B000B245FEFFB245FEFFB245FEFFB245FEFF70
:1000C000B245FEFFB245FEFFB245FEFFB245FEFF60
:1000D000B245FEFFB245FEFFB245FEFFB245FEFF50
:1000E000B245FEFFB245FEFFB245FEFFB245FEFF40
:1000F000B245FEFFB245FEFFB245FEFFB245FEFF30
:100100004C45FEFF6245FEFFB245FEFFB245FEFFD5
:10011000B245FEFFB245FEFFB245FEFFB245FEFF0F
:10012000B245FEFFA845FEFFB245FEFFB245FEFF09
:100130005A43FEFF1244FEFFB245FEFFB245FEFFEA
:100140004844FEFFB245FEFFA044FEFFB245FEFF5D
:10015000B245FEFFCE44FEFFC048FEFF1449FEFF3D
:10016000C848FEFF1449FEFF1449FEFF1449FEFF74
:100170001449FEFFBA47FEFF1449FEFF1449FEFF73
:10018000D447FEFFE047FEFF1449FEFFF247FEFFA3
:10019000FE47FEFFFE47FEFFFE47FEFFFE47FEFF57
:1001A000FE47FEFFFE47FEFFFE47FEFFFE47FEFF47
:1001B000FE47FEFF1449FEFF1449FEFF1449FEFFEF
:1001C0001449FEFF1449FEFF1449FEFF1449FEFFC7
:1001D0001449FEFF1449FEFF1449FEFF1449FEFFB7
:1001E0001449FEFF1449FEFF1449FEFF1449FEFFA7
:1001F0001449FEFF1449FEFF1449FEFF1449FEFF97
:100200001449FEFF1449FEFF1449FEFF1449FEFF86
:100210001449FEFF1449FEFF1449FEFF1449FEFF76
:100220001449FEFF1449FEFF1449FEFF1449FEFF66
:100230001449FEFF1449FEFF1449FEFF1449FEFF56
:100240001449FEFF1449FEFF1449FEFF1449FEFF46
:100250001449FEFF1449FEFF3248FEFF6048FEFFCE
:100260001449FEFF1449FEFF1449FEFF1449FEFF26
:100270001449FEFF1449FEFF1449FEFFB648FEFF75
:100280001449FEFF1449FEFF1846FEFF1247FEFF09
:100290001449FEFF1449FEFF8447FEFF1449FEFF88
:1002A000AA47FEFF1449FEFF1449FEFF0E49FEFF58
:1002B000000102020303030304040404040404040D
:1002C00005050505050505050505050505050505DE
:1002D00006060606060606060606060606060606BE
:1002E00006060606060606060606060606060606AE
:1002F000070707070707070707070707070707078E
:10030000070707070707070707070707070707077D
:10031000070707070707070707070707070707076D
:10032000070707070707070707070707070707075D
:10033000080808080808080808080808080808083D
:10034000080808080808080808080808080808082D
:10035000080808080808080808080808080808081D
:10036000080808080808080808080808080808080D
:1003700008080808080808080808080808080808FD
:1003800008080808080808080808080808080808ED
:1003900008080808080808080808080808080808DD
:1003A00008080808080808080808080808080808CD
:1003B000546D725100000000546D7220537663003A
:1003C000286E756C6C2900004572726F7220696E20
:1003D0002051756575654F76657277726974652011
:1003E0007461736B73200D0A000000006D69616F0A
:1003F000750A00006D69616F75320A0068756E6775
:1004000072790A0054696D65723200004368656351
:100410006B54696D65720000514F76657200000083
:100420001000000000000000017A5200017C010170
:100430001B0D02001000000018000000C84CFEFF59
:100440008A03000000000000100000002C000000E3
:100450003E50FEFF5E0300000000000010000000A0
:10046000400000008853FEFF54030000000000001D
:0C04E400FC8F0100090000000100000076
:040000058000004037
:00000001FF
